:100000000C9414010C9431010C9431010C943101C5
:100010000C9431010C9431010C9431010C94310198
:100020000C9431010C9431010C94911B0C94631CC1
:100030000C9477160C9431010C9431010C9431011D
:100040000C9431010C9431010C9431010C94310168
:100050000C9431010C94FF160C9431010C94310175
:100060000C9431010C9431010C9431010C94310148
:100070000C9431010C9431010C9431010C94310138
:100080000C9431010C9431010C9431010C94310128
:100090000C9431010C9431010C9431010C94310118
:1000A0000C9431010C9431010C9431018E038E03B8
:1000B000BA03BA0322044004580558054B04E4046B
:1000C000F504F504D01CF71CEF1DF71CEF1D431DB4
:1000D000661DEF1DBD1DCC1D0151AA00A900AC007D
:1000E000AE00AB000100A75DA85D000000000000AD
:1000F0001603730069007800730068006F006F00DA
:100100007400650072000000120362007000690054
:100110007000680061006E007900000004030904AB
:1001200009023B00020100A0FA09040000010301DA
:100130000100092111010001224000070581030887
:100140000001090401000103000000092111010060
:1001500001227B000705820320000112010002003A
:10016000000008EDFE6666010001020001050109BC
:1001700002A10185020901A100050919012908153B
:100180000025019508750181020501093009311525
:1001900081257F95027508810609381581257F958F
:1001A0000175088106050C0A38021581257F950125
:1001B00075088106C0C005010980A10185031901E8
:1001C0002AB700150126B700950175108100C005FA
:1001D0000C0901A101850419012AA002150126A01C
:1001E00002950175108100C005010906A1010507EE
:1001F00019E029E71500250195087501810295018F
:10020000750881010507190029FF150026FF0095D3
:1002100006750881000508190129059505750191E4
:1002200002950175039101C011241FBECFEFDAE0E2
:10023000DEBFCDBF11E0A0E0B1E0E4E4FDE302C029
:1002400005900D92A238B107D9F722E0A2E8B1E0FB
:1002500001C01D92AA32B207E1F70E94BF100C94B0
:10026000A01E0C9400009C01FB018281882319F1DF
:10027000273AFDE53F0721F0283A3D4571F0089502
:10028000269A2E9A3F9A479A509A589A259A2D9ACA
:10029000579A5F9A279A2F9A0CC026982E983F98C3
:1002A00047985098589825982D9857985F98279870
:1002B0002F9880E0089581E00895269A2E9A3F9A1B
:1002C000479A509A589A259A2D9A579A5F9A279A40
:1002D0002F9A089581E008950C94330108950C94A9
:1002E0006E011F93CF93DF9300D000D01F92CDB744
:1002F000DEB749835A836B833091850189819A8166
:10030000311114C0662359F0222349F00E94950749
:10031000182F682F89819A810E943E0703C00E948E
:100320006907182F69817A81812F04C00E9495077F
:1003300069817A810F900F900F900F900F90DF914D
:10034000CF911F910C94B00EFC01262F408151815A
:100350006281738184810C94710181E00895CF934F
:10036000DF93EC0160E00E94A401BE01DF91CF9118
:100370000C946F010C94D50F0C94D30F08950E9428
:10038000E8050E94BE012FEF84E39CE021508040ED
:100390009040E1F700C000000C9425170F931F93C5
:1003A000CF93DF938C0161E00E94A401EC01B801BE
:1003B0000E946C018823F1F1B801CE010E94411521
:1003C0008823C1F1B801CE010E945513882391F111
:1003D000B801CE010E949D14882361F1F801828149
:1003E000882309F1CB358DE5D807C1F050F4C1154C
:1003F000FCE5DF0781F0CF3DDC45A9F40E94C60C87
:1004000019C0CC35EDE5DE0761F0CD35DD4559F499
:100410000E940F0C08C00E94BF010CC00E94180C63
:1004200002C00E941B0CC801DF91CF911F910F9158
:100430000C946A0180E0DF91CF911F910F91089594
:100440000E9458160C9439020E943C020C945E16CD
:1004500008950C94280281E008950C942B020895CD
:10046000CF93C82F0E9429028C2F0E942D02CF917A
:10047000089580E00C9430020E949D150C94300287
:100480000E949D1590918401891721F08093840129
:100490000C9430020895CF93DF93CDB7DEB72B973E
:1004A0000FB6F894DEBF0FBECDBF4F835887698764
:1004B0007A878B8761110E945B0B9E012F5F3F4FF4
:1004C00086E0F90111928A95E9F785E0FE013796F9
:1004D000D90101900D928A95E1F789819A814C8129
:1004E0005D81452B31F09F3F31F491E08F3F19F44E
:1004F00003C091E001C090E090FF09C049815A819A
:100500006B817C818D819E810E947C0A05C0C9011E
:100510000E94AD018111F2CF2B960FB6F894DEBF89
:100520000FBECDBFDF91CF910895FC0180819181F5
:100530000E94D7070895CF93882309F450C0C82F8D
:100540008CEF8C0F813AD0F46C2F80910201909146
:1005500003010E94FA15882349F06C2F8091020153
:10056000909103010E9432160E947D0B6C2F8091A6
:100570000201909103010E9430160CC080E28C0FA2
:10058000883058F4C77081E001C0880FCA95EAF737
:100590000E943E0BCF910C947D0BEBE5EC0FE3300A
:1005A00040F4F0E0E95BFE4F808190E0CF910C9445
:1005B000C215E8E5EC0FE73150F4F0E0EE0FFF1F55
:1005C000E75EFE4F80819181CF910C94D815CD3E8E
:1005D00030F08C2F0E944411CF910C941612CF91C1
:1005E0000895882389F19CEF980F913A40F4682F81
:1005F00080910201909103010E9432160DC090E299
:10060000980F983058F4877091E001C0990F8A953F
:10061000EAF7892F0E94440B0C947D0B9BE5980F01
:10062000933020F480E090E00C94C21598E5980F88
:10063000973120F480E090E00C94D8158D3E20F0A6
:100640000E949F110C94161208951F93CF93DF936D
:10065000182FEB010E949B02209741F08FE99FE049
:100660000197F1F700C000002197F6CF812FDF91AD
:10067000CF911F910C94F102893319F060E070E082
:1006800002C060E570E00C942503882321F00E94ED
:100690003E0B0C947D0B0895882321F00E94440B9F
:1006A0000C947D0B0895CF92DF92EF92FF920F93FF
:1006B0001F93CF93DF937C01D62FC72FFC011281AC
:1006C000058102950F700E94340B8823B9F0112325
:1006D000A9F08C2F807F803421F080E28D0F88304C
:1006E00068F08091140282FD09C082E00E94DD0B57
:1006F0000E94340B91E0D82ED92601C0D12CCC2EEB
:10070000C2948FE0C8228C2D90E08C30910508F0C7
:10071000CFC1FC01EA5AFF4F0C94371E8C2F807F0B
:10072000CF70882311F0C295C07F112399F0CC239C
:1007300009F4AAC180E28D0F883010F0D11104C0F5
:100740008C2F0E943E0B03C08C2F0E944E0B0E94E8
:100750007D0B9AC18D2F0E94F102CC2309F4A8C110
:1007600080E28D0F883038F1DD2329F18C2F0E9433
:10077000540B24C08C2F807FCF70803211F0C29533
:10078000C07FDD2319F0D130A1F13DC0809114026A
:1007900082FF17C0112349F0CC2329F08C2F0E942F
:1007A0003E0B0E947D0B80E070C180E00E94F10250
:1007B000CC2309F47DC18C2F0E94440B0E947D0B39
:1007C00077C1112371F0002341F0013031F40E9410
:1007D0005E0B8C2B0E94660B6BC10E945E0B8C2BF8
:1007E0001DC0002319F0013009F462C10E94730B8F
:1007F00025C0112321F0063008F05AC10EC0053083
:1008000008F056C11BC0112361F0002331F0F7013D
:10081000858180FF39C18F7085838C2F0E944503AD
:1008200047C1002359F0D93309F03FC1FFEF07EE6C
:1008300013E0F15000401040E1F735C18C2F0E94C9
:100840004C0336C18C2F86958695837019F08130C4
:1008500061F02EC1112321F08D2F9C2F937002C0C7
:1008600080E090E00E94C2152BC1112321F08D2F52
:100870009C2F937002C080E090E00E94D81520C1A8
:100880008D2F112319F00E94441102C00E949F1164
:100890000E94161215C18C2F837009F047C01111E8
:1008A0000BC12D2F229526952770220F220F6D2F19
:1008B0006F70862F90E0A0E0B0E0022E04C0880F99
:1008C000991FAA1FBB1F0A94D2F7D4FF10C04FE094
:1008D00050E060E070E004C0440F551F661F771FB2
:1008E0002A95D2F7409550956095709503C040E0E9
:1008F00050E0BA01C695C695C3708A019B01082BCA
:10090000192B2A2B3B2BC901B801C23049F058F4EE
:10091000C13019F00E945406CFC00E944206CCC0DC
:100920000E946606C9C00E944006C6C0112319F085
:100930008C2F817001C08695882309F4BDC02D2FAE
:10094000229526952770220F220F6D2F6F70862F0C
:1009500090E0A0E0B0E0022E04C0880F991FAA1F0B
:10096000BB1F0A94D2F7D4FF10C04FE050E060E004
:1009700070E004C0440F551F661F771F2A95D2F7F9
:10098000409550956095709503C040E050E0BA01E5
:10099000C695C695C3708A019B01082B192B2A2B7B
:1009A0003B2BC901B801C23049F058F4C13019F0ED
:1009B0000E94190781C00E9407077EC00E942B0772
:1009C0007BC00E947A0678C0CF70112339F08C2F3B
:1009D0000E94A0068D2F0E9445036EC08D2F0E949D
:1009E0004C038C2F0E94C10667C0D23F21F128F42E
:1009F000D03F41F0D13FC1F043C0D33F19F1D43FC4
:100A000079F03EC0112341F0053008F051C08C2F21
:100A10008F710E94E6064CC0063008F049C0F7CF3F
:100A20008091140282FF18C0112339F08C2F8F712E
:100A30000E94A0063DC01123C9F38C2F8F710E9424
:100A4000C10636C0112329F08C2F8F710E948B06AE
:100A50002FC00E9486062CC0112349F0CF718C2F25
:100A60000E94A00663E08C2F0E94C20B21C081E08F
:100A70000E94DD0B0230E0F082E00E94DD0B18C026
:100A8000112331F0002391F28D2F0E949B0210C0A0
:100A9000002399F2D93349F41FEF27EE33E01150C8
:100AA00020403040E1F700C000008D2F0E94F1028D
:100AB00088EF8C0D843020F40E949D150E94300236
:100AC000DD20C9F00E94300B80FD15C0F7011282B5
:100AD0000E942A0B0E94A006C7010E949C050E944A
:100AE0002A0BDF91CF911F910F91FF90EF90DF9034
:100AF000CF900C94C106DF91CF911F910F91FF9081
:100B0000EF90DF90CF9008950F931F93CF93DF93D3
:100B1000EC01688179818A810E94E2078C010E9440
:100B20003D070E942E06B801CE010E945303DF91BB
:100B3000CF911F910F910895CF93DF93EC0198818E
:100B400089812B813C81232B31F08F3F31F481E06F
:100B50009F3F19F403C081E001C080E080FD1DC00B
:100B6000CE010E94CE01811110C00E94340B882357
:100B7000A1F08A81882389F08091140282FD0DC042
:100B800082E0DF91CF910C94DD0BCE010E948405B1
:100B9000CE01DF91CF910C94AF01DF91CF910895F9
:100BA00080E090E00E94C21580E090E00E94D8159D
:100BB0000E945B0B0E947D0B0E9447130C9416123F
:100BC00080910201909103010E9434160C94D0058B
:100BD0000E944B0B0C94E00592959F70963079F033
:100BE00010F4925001C09A50923068F4803F69F03E
:100BF00018F4883E40F409C0843F29F406C0883EBA
:100C000020F0813F11F080E0089581E00895FC011B
:100C1000808191810E94D7070E94EC050895CF93AF
:100C2000DF9300D000D01F92CDB7DEB70F900F90AA
:100C30000F900F900F90DF91CF910895CF93DF9396
:100C400000D000D000D0CDB7DEB726960FB6F8940E
:100C5000DEBF0FBECDBFDF91CF91089508950895F7
:100C60000C942F060C9430060E94320660938F017C
:100C70007093900180939101909392010C94D00510
:100C80000C9434060F931F9300918F0110919001E3
:100C90002091910130919201602B712B822B932B2B
:100CA0001F910F910C9434060F931F9300918F01A5
:100CB0001091900120919101309192016023712354
:100CC000822393231F910F910C9434060F931F934B
:100CD00000918F011091900120919101309192012A
:100CE00060277127822793271F910F910C94340658
:100CF0000C942F060E94780660938B0170938C01F0
:100D000080938D0190938E010C94D00560E070E08B
:100D1000CB010C947A060F931F9341E050E060E002
:100D200070E08A019B0104C0000F111F221F331FB6
:100D30008A95D2F7C901B8011F910F910C947A06D8
:100D40000F931F9341E050E060E070E004C0440F57
:100D5000551F661F771F8A95D2F780918B0190915E
:100D60008C01A0918D01B0918E018A019B01082B0D
:100D7000192B2A2B3B2BC901B8011F910F910C9401
:100D80007A060F931F9341E050E060E070E004C0EA
:100D9000440F551F661F771F8A95D2F740955095CF
:100DA0006095709580918B0190918C01A0918D013F
:100DB000B0918E018A019B01082319232A233B232A
:100DC000C901B8011F910F910C947A060F931F93DC
:100DD00041E050E060E070E004C0440F551F661F22
:100DE000771F8A95D2F780918B0190918C01A09109
:100DF0008D01B0918E018A019B01082719272A27AE
:100E00003B27C901B8011F910F910C947A060F93EB
:100E10001F9300918B0110918C0120918D013091D5
:100E20008E01602B712B822B932B1F910F910C94B1
:100E30007A060F931F9300918B0110918C012091E2
:100E40008D0130918E0160237123822393231F91A2
:100E50000F910C947A060F931F9300918B011091C0
:100E60008C0120918D0130918E016027712782279E
:100E700093271F910F910C947A060895292F220F22
:100E8000920F890FE82FE695E695E695877051E079
:100E900001C0550F8A95EAF785E0E89FF00111241B
:100EA000EA57FE4F20E030E070E04081CB01022E97
:100EB00002C0969587950A94E2F781708195842700
:100EC0008523842781932F5F3F4F2530310569F7B4
:100ED0000895292F220F920F890F682F6695669526
:100EE0006695982F977085E0689FB001112440E0C7
:100EF00050E080E0FB01E40FF51FEA57FE4F208130
:100F000030E0092E02C0369527950A94E2F7217049
:100F10003327042E01C0220F0A94EAF7822B4F5F79
:100F20005F4F4530510531F70895BF92CF92DF9260
:100F3000EF92FF920F931F93CF93DF938C01C0909A
:100F40008B01D0908C01E0908D01F0908E0180910A
:100F50008F0190919001A0919101B0919201C82AC6
:100F6000D92AEA2AFB2ACFE1D0E0D701C6010C2E0C
:100F700004C0B695A795979587950A94D2F780FDFA
:100F800004C0219790F7B12C07C0BC2EB8018C2F5C
:100F90000E94C60E0197A9F38B2DDF91CF911F916F
:100FA0000F91FF90EF90DF90CF90BF900895CF9377
:100FB000DF93EC010E949507BE010E94C60EDF91EF
:100FC000CF9108951F93CF93DF93EB01909185010B
:100FD000992321F0CB010E94D70713C0882349F041
:100FE000CB010E949507182F682FCE010E943E0763
:100FF00004C0CB010E946907182FBE01812F0E94F7
:10100000C60EDF91CF911F9108951F93CF93DF9369
:10101000C091930116E080919401C81799F0D0E037
:101020001C9FF0011D9FF00D1124EB56FE4F4081D7
:10103000518162817381848195810E941E0621966F
:10104000C770E9CFDF91CF911F9108954091C501FD
:101050005091C6016091C7017091C8018091C9018A
:101060009091CA010C941E06EF92FF920F931F936A
:10107000CF93DF938091CA0182958F7009F065C08C
:101080008091C701882309F460C080919301F0909A
:1010900094011091C5010091C6016091C801709141
:1010A000C90191E01F3F09F090E0C0910001D0918B
:1010B0000101292F96E0E92E8F1509F446C061152C
:1010C000710521F00F3F21F030E003C031E001C095
:1010D000322F90E030FD36C0E89EF001E99EF00D21
:1010E0001124DF01AB56BE4F11963C91119730137E
:1010F00029C03C91311326C012963C9112973111B0
:1011000021C013964D915C911497461B570B4C17B9
:101110005D07C0F48091CA018F7080618093CA011D
:10112000E656FE4F80818F708061808385EC91E070
:101130000E949C05DF91CF911F910F91FF90EF903E
:101140000C94050801968770B7CFDF91CF911F915E
:101150000F91FF90EF9008959F92AF92BF92CF9220
:10116000DF92EF92FF920F931F93CF93DF93CDB750
:10117000DEB761970FB6F894DEBF0FBECDBF8C010E
:1011800085E0F801DE011D9601900D928A95E1F748
:10119000D8011296EC909091C501E091C601209182
:1011A000C8013091C9012115310531F0EF3F31F40B
:1011B00081E09F3F19F403C081E001C080E0B82FB7
:1011C000B1709B2E80FD47C1D8014C9111965C9166
:1011D00011971396AD90BC90149785ECC82E81E0C2
:1011E000D82EF090C701B501621B730B209100014E
:1011F00030910101FF2009F4D9C08091CA01621722
:10120000730708F095C0282F207F09F052C05E13A5
:1012100013C0491311C0FE2CE1100EC08F70806105
:101220008093CA010E942608C6010E949C058091F5
:10123000CA01F80185834DC1AB2831F05F3F31F41D
:1012400081E04F3F19F403C081E001C080E080FDE0
:1012500003C081E08E2502C080E090E0F82FF1709D
:10126000FF2E80FF1CC0809193012091940136E0F5
:10127000821709F40BC190E0389FF001399FF00DFF
:101280001124EB56FE4F6181561306C06081461350
:1012900003C06281E61203C001968770E9CFFE2C7D
:1012A000EE2009F416C18091CA0181608093CA01C1
:1012B00054C05E1306C0491304C0E11002C0F80117
:1012C00099C0C8010E940706882361F1EE2051F100
:1012D0002091CA01822F82958F7090E0029774F05E
:1012E0008091C5019091C60198878F831986BB862E
:1012F000AA862C87CE0107960E949C0586E0F801FD
:10130000A5ECB1E001900D928A95E1F70E943408B6
:101310000E9426080AC05E1711F1C8010E94070644
:1013200081112CC0C8010E949C05FF24F394D1C0F8
:10133000282F207F81F77A2DB98AA88A6E2D898976
:101340000E940F0685EC91E00E949C0586E0D60184
:101350001D928A95E9F70E942608F12CBAC049131C
:10136000DCCFE110DACFF8018583C8010E949C052B
:1013700086E0D6011D928A95E9F7ABC0EE2091F286
:101380002091CA01822F82958F7090E002970CF411
:10139000B5CF8091C5019091C6019A8389831B8244
:1013A000BD82AC822E83CE010196A6CF6217730751
:1013B00008F044C0FE2CEE2009F4B4CF5E1330C018
:1013C00049132EC02091CA0120FD21C0822F829591
:1013D0008F70482F50E041155105C9F0F801258361
:1013E0004F30510541F08F5F982F9295907F822F5B
:1013F0008F70892B8583C8010E949C0586E0F801C7
:10140000A5ECB1E001900D928A95E1F73CC086E031
:10141000F801A5ECB1E001900D928A95E1F759C071
:10142000C8010E940706811169CF8091CA018160BD
:101430008093CA01C8010E949C054BC07A2DB98ACD
:10144000A88A6E2D89890E940F0686E0D6011D921A
:101450008A95E9F718C0EE2009F464CFC8010E940C
:101460000706F82E882309F45DCF86E0F801A5EC85
:10147000B1E001900D928A95E1F785EC91E00E9430
:1014800095020E9434080E94260823C04D875E877B
:101490008D859E850E94D707292F22952F70223097
:1014A00028F49F7039F0811105C00BC0243028F456
:1014B0009F7049F4805E883020F0C8010E949C052E
:1014C0009F2CF92C06C0D80115969C91907F91F71E
:1014D000F8CF8F2D61960FB6F894DEBF0FBECDBF4B
:1014E000DF91CF911F910F91FF90EF90DF90CF9000
:1014F000BF90AF909F9008951F93CF93DF93CDB788
:10150000DEB72C970FB6F894DEBF0FBECDBF4F836A
:10151000588769877A878B879C87CE0107960E94B8
:10152000AC088823D1F09F8188852A853B85232BB1
:1015300031F08F3F31F481E09F3F19F403C081E027
:1015400001C080E080FD47C04F81588569857A855C
:101550008B859C850E941E063EC086E0FE01379664
:10156000DE01119601900D928A95E1F7FF81E885E1
:101570006A857B856115710531F0EF3F31F481E0BB
:10158000FF3F19F403C081E001C080E080FD23C06B
:101590002091940130E0C90101968770992740910C
:1015A000930150E084179507F1F1F983EA837D8375
:1015B0006C8396E0929FD001939FB00D1124AB569F
:1015C000BE4FFE01319601900D929A95E1F78093FE
:1015D00094010E94050816E0809193019091940176
:1015E000891771F1189FC00111248B569E4F0E94DC
:1015F000AC08882329F1E09193011E9FF00111248A
:10160000EB56FE4F408151816281738184819581C7
:101610000E941E068091930190E0019687709927A1
:1016200080939301D9CF0E94E80510929401109203
:101630009301E5ECF1E086E0DF011D928A95E9F780
:101640002C960FB6F894DEBF0FBECDBFDF91CF91C1
:101650001F9108958091D30185958595859508956D
:101660008091D301877008959091D301977081E0A4
:1016700009F480E008958091DE0108959091DE01E3
:10168000892B8093DE01089580959091DE01892356
:101690008093DE0108951092DE0108959091DD019E
:1016A000892B8093DD01089580959091DD01892338
:1016B0008093DD0108951092DD0108958091D40199
:1016C000089508950C94610B0C94620B9091140290
:1016D00092FD08C09091D401981721F08093D40115
:1016E0000C94640B08958091D401882329F0109202
:1016F000D40180E00C94640B0895CF93DF93E091C4
:101700000201F09103018091DE018083E0910201EA
:10171000F091030190818091DD01892B808380917C
:10172000D401882381F0E0910201F09103019081BE
:10173000892B808380910201909103010E94EE1514
:1017400081110E94730BC0910201D091030148E006
:1017500050E06BEC71E0CE010E94511E892B69F0C4
:1017600088E0FE01ABECB1E001900D928A95E1F7C3
:10177000CE01DF91CF910C94A915DF91CF910895FF
:101780000C94610B9091140292FD10C098E0899F17
:1017900090011124262B2093D3010E94A006809152
:1017A000D3018595859585950C94C00B0C94A00666
:1017B0001092D30180E00C94C00B2091D30180954E
:1017C00082238093D301982F977099F430E0482FAB
:1017D000082E000C550B2417350759F09091140270
:1017E00092FD07C08595859585950E94C1060C944C
:1017F000D80B08959091140292FB222720F9281704
:1018000069F080FB92F990931402809113029091F9
:1018100014020E94420C82E00C94DD0B089580912A
:10182000140282FB882780F991E089270C94FA0B37
:1018300081E00C94FA0B80E00C94FA0B80E090E0CD
:101840000E94661E21E0893E9E4F09F020E0822F13
:10185000089582E090E00C945E1E83E090E00C948A
:101860005E1ECF9384E090E00E945E1EC82F82E24D
:1018700090E00E945E1E2C2F30E0A901582BCA0177
:10188000CF910895CF93C92F682F84E090E00E94F4
:101890006C1E6C2F82E290E0CF910C946C1EAB0119
:1018A000BC018FE090E00C947E1EAB01BC0183E193
:1018B00090E00C947E1E60E070E0CB010C94550C1F
:1018C00060E070E0CB010E944F0C0C945B0C69EE61
:1018D0007EEF80E090E00E948A1E60E082E090E06F
:1018E0000E946C1E60E083E090E00E946C1E1092EB
:1018F0008F0110929001109291011092920160E07C
:1019000084E090E00E946C1E60E082E290E00E9421
:101910006C1E60E085E090E00E946C1E60E086E056
:1019200090E00E946C1E6FEF87E090E00E946C1EBA
:1019300040E050E0BA0188E090E00E947E1E60E046
:101940008DE090E00E946C1E40E050E0BA0188E11A
:1019500090E00E947E1E60E087E190E00E946C1E95
:1019600040E050E0BA018CE190E00E947E1E60E011
:1019700070E080E290E00E948A1E40E050E0BA01F0
:1019800088E190E00E947E1E0C94600C0C94670C21
:10199000682F8EE090E00C946C1E0E94E416609319
:1019A000E5017093E6018093E7019093E80160936D
:1019B000E1017093E2018093E3019093E4010895C3
:1019C00085B7806885BF85B7806885BF089581E049
:1019D00008950C94E70C08950C94EB0C0C94EB0C0C
:1019E0000C94EE0C0C94EB0C0C94F20C0C94EB0C91
:1019F0000E94E00C82EA9FE00E9493150E94F60C80
:101A00000C94F40C0E94EC0C0C94EB0C0E94A50FAF
:101A10000C942F020E94CF160E9435100E94060DD2
:101A20000C94F00C8F929F92AF92BF92CF92DF9264
:101A3000EF92FF920F931F93CF93DF93CDB7DEB753
:101A40002A970FB6F894DEBF0FBECDBF0E94441098
:101A5000982E81110E94CD0C8FEDA82E81E0B82E1A
:101A600000E010E0802E802F0E94C90FD82EF501D3
:101A7000C1905F01C826B1F40F5F1F4F02301105FE
:101A800089F78FEF89838A831B820E94D816816031
:101A9000782F9D838C8349815A816B818D810E942F
:101AA0004B022FC08091E90181FD0E94CF0FE12CF4
:101AB000FF24F3948C2D8F21F1F00E94E90C8823F0
:101AC00099F0EE828F82DF2081E009F480E0888740
:101AD0000E94D8168160782F9A8789874E815F810E
:101AE00068858A850E944B02F801E152FE4F808191
:101AF000F826F08206C0E394FF0CF3E0EF12DACF91
:101B0000BBCF81E0911001C080E02A960FB6F89417
:101B1000DEBF0FBECDBFDF91CF911F910F91FF9020
:101B2000EF90DF90CF90BF90AF909F908F900895EF
:101B30000E94120D0E9434120C944002CF93DF9346
:101B40000E94CB0EEC01811521E5920708F045C0FB
:101B5000811530E5930708F094C0883E910528F57B
:101B6000803E910508F0F8C0883A910570F4853AF6
:101B7000910508F07CC08130910509F475C008F426
:101B8000E8C0049708F0E8C0E4C08F3B910508F076
:101B9000E0C0C85AD0E0CC0FDD1FC65BDE4F099015
:101BA000D881C02DCE019464D8C0811540E294073D
:101BB00058F4811551E0950708F0CEC08D3E91058F
:101BC00008F4C7C09065C9C0C11580E4D80708F4FF
:101BD000C0C0DF70CE01906AC0C0811525E59207B4
:101BE000A8F4811534E5930708F095C0811543E505
:101BF000940708F07BC0811552E5950708F061C095
:101C0000D82FCC27CE01816F906AA7C0C11589E576
:101C1000D807A0F4C11528E5D20708F082C0C11585
:101C200036E5D30708F095C08C2F0E945F0F8F71A7
:101C300090E0D82FCC27CE0190628FC0C1154AE525
:101C4000D40708F474C0CE0190568115904208F074
:101C500080C08D2F8F710E945F0FDD27D0628F7142
:101C6000AE01582BCA0179C081E090E076C0C55A18
:101C7000D0E0C858DE4F8881C82FD0E0CE019064F4
:101C80006CC074E0969587957A95E1F7282F2370BC
:101C90003C2F337081E090E002C0880F991F3A9585
:101CA000E2F79C68AC01522B9A019C2F9F7096958D
:101CB000969550E2959FE0011124C9018C2B9D2B34
:101CC0004CC08370992721E030E002C0220F331FFF
:101CD0008A95E2F79C2F9695969580E2989FE00171
:101CE0001124C22BD32BCE019C6837C08370992757
:101CF00021E030E002C0220F331F8A95E2F79C2FCB
:101D00009695969540E2949FE0011124C22BD32B27
:101D1000CE019A6822C0D82FCC27CE01846F906A5A
:101D20001CC0DC2FCC27CE01806F906A16C08C2F90
:101D30008F700E945F0F94E0D695C7959A95E1F752
:101D4000CF70D0E0DC2FCC27D0699E01282BC901B1
:101D500004C080E090E001C0CE01DF91CF910895F2
:101D6000272F30E0F901EE0FFF1F2E0F3F1FF90163
:101D700096E0899FE00DF11D1124E60FF11DEE0F95
:101D8000FF1FE852FF4F8591949108950E94B00E75
:101D90000E949E0D08958238910569F1B0F4813357
:101DA000910509F46DC048F48932910509F463C0C6
:101DB0008A32910509F469C008958533910509F4C3
:101DC00055C089339105B9F00895833E910569F1B5
:101DD00038F4803E9105B1F0823E910509F10895F5
:101DE000863E9105A9F1873E9105B9F1843E9105A2
:101DF00009F064C023C02091130220FD4FC021FDD3
:101E00004DC008958091130280FD44C0809114025A
:101E100080FF44C08091130284FD42C083EE4DC018
:101E20008091130282FF38C0F5CF8091130282FDAA
:101E300033C08091140280FD31C0ECCF8091140238
:101E400081FF32C08091130284FD2AC087EE35C025
:101E50008091130283FF26C0F5CF8091130283FD8A
:101E600021C08091140281FD1FC0ECCF809113022C
:101E700085FD1CC01DC08091130285FD19C016C0D0
:101E80008091130286FD16C017C08091130286FD53
:101E900013C010C089E311C082EE0FC080EE0DC0E8
:101EA00080E00BC086EE09C084EE07C089E205C061
:101EB00085E303C08AE201C081E390E00895909138
:101EC000130292FF0DC0282F2871283019F4877F44
:101ED000846006C0282F2471243011F48B7F886021
:101EE00093FF0DC0282F2871283119F4877E846153
:101EF00006C0282F2471243111F48B7E8861209133
:101F0000140220FF0DC0382F3871383019F4877F44
:101F1000816006C0382F3171313011F48E7F8860B6
:101F200021FF0DC0282F2871283119F4877E816187
:101F300006C0282F2171213111F48E7E886194FD15
:101F4000877E089580E0089508950E941E0C8111F7
:101F500002C00E94C60C0E94290C8093E9010E94D5
:101F6000310C90931402809313020E94A40F0E94DC
:101F70002D0C682F70E080E090E00E944006609198
:101F80008B0170918C0180918D0190918E010C9448
:101F90007806E82FF0E0E95EFD4F8081089508950E
:101FA00008950C94D00F0C94D10F0C945D01CF9335
:101FB000DF934BE751E0A1E0B0E020E030E0FA0130
:101FC000E20FF31F80818F3FA1F0E82FE295EF70C1
:101FD000F0E061A18F70ED0102C0CC0FDD1F8A958A
:101FE000E2F7CE019C2F9095962391A392A1892B85
:101FF00082A32F5F3F4F2330310509F74D5F5F4FBD
:10200000D1E041385D07C9F6DF91CF910895CF93B4
:10201000DF93DC01462F50E083E0689FF00111243C
:10202000E558FE4F73E081E060E091919F3F99F0A9
:10203000C92FC295CF70D0E028A130E09F7002C0B8
:10204000359527959A95E2F720FD02C0282F02C00A
:1020500020E030E0622B880F715039F7FD01E40F6A
:10206000F51F6083DF91CF9108950E94D70F1092E2
:10207000180210921702109216021092150282E0B6
:102080000E947C100C94BA011F93CF93DF9300D071
:10209000CDB7DEB71A82198260E0CE0101960E94A8
:1020A000071061E0CE0101960E94071042E050E067
:1020B000BE016F5F7F4F85E192E00E94511E11E0EB
:1020C000009709F410E0892B31F089819A8190936F
:1020D000160280931502212F42E067E172E085E14C
:1020E00092E00E947D100E94BC01812F0F900F9002
:1020F000DF91CF911F9108950895FF920F931F9341
:10210000CF93DF938C01F62ED72FC42F222349F0D3
:1021100081E08093EC010E94D8169093EB018093AC
:10212000EA018091EC018823C1F08091EA0190914D
:10213000EB010E94F016059780F0EF2DFD2FD801DE
:102140004C2F50E0CD01801B910B841795071CF498
:102150008D918193F7CF1092EC01DF91CF911F9178
:102160000F91FF9008950E94E9180E940A0D0C94A7
:10217000F5180E94F9180E94980D0C9413190E94EA
:1021800076160E94D0180E94F80C0E94B3100E948C
:10219000B9100E94020DFBCF8091F30180FF06C0B1
:1021A0006091090170E0660F771F26C081FF04C0AF
:1021B0006091090184E005C082FF07C060910901B8
:1021C00088E0689FB001112417C09091F201992313
:1021D000D1F060910801961788F72091090188E0F5
:1021E000289F90011124929FA001939F500D1124CC
:1021F00070E0CA010E94231E6038710540F4611529
:10220000710519F406C068E070E0862F08958FE725
:10221000089581E008958091F30180FF08C06091E6
:10222000050170E0759567957595679521C081FFEB
:1022300006C06091050170E07595679519C082FF31
:1022400004C06091050170E010C09091F1019923E4
:1022500099F0609104019617A0F780910501899F7C
:10226000C001112470E00E94231E6038710540F403
:102270006115710519F406C061E070E0862F0895BC
:102280008FE7089581E008958D3E21F40E94CC10DF
:10229000819504C08E3E29F40E94CC108093F701F2
:1022A00008958F3E21F40E94CC10819504C0803F98
:1022B00029F40E94CC108093F6010895893F19F407
:1022C0000E940B1105C08A3F31F40E940B118195C9
:1022D0008093F80108958B3F21F40E940B118195A2
:1022E00004C08C3F29F40E940B118093F9010895DA
:1022F0009FE0980F983078F421E030E0A90102C007
:10230000440F551F9A95E2F7CA019091F501892B68
:102310008093F50108958D3F21F48091F301816050
:102320000BC08E3F21F48091F301826005C08F3F86
:1023300029F48091F30184608093F30108958D3E28
:1023400039F49091F70197FF35C01092F70159C009
:102350008E3E29F49091F7011916BCF32BC0909191
:10236000F6018F3E29F497FF25C01092F60149C06F
:10237000803F19F41916CCF31DC09091F801893FE4
:1023800029F41916BCF41092F8013BC08A3F19F4E5
:1023900097FF10C0F8CF8B3F39F49091F90197FF68
:1023A00009C01092F9012DC08C3F21F49091F901E0
:1023B0001916BCF39FE0980F983080F421E030E0CC
:1023C000A90102C0440F551F9A95E2F7CA018095F2
:1023D0009091F50189238093F50113C08D3F21F47D
:1023E0008091F3018E7F0BC08E3F21F48091F30129
:1023F0008D7F05C08F3F29F48091F3018B7F8093FF
:10240000F3018091F601811106C08091F7018111DD
:1024100002C01092F2018091F801811106C08091F2
:10242000F901811102C01092F10108950E94D8169D
:102430002091F601211104C02091F701222321F0FF
:102440009093F0018093EF012091F801211104C0D5
:102450002091F901222321F09093EE018093ED0168
:1024600084EF91E00C94B415EF92FF920F931F93B9
:10247000CF93DF9300D000D000D0CDB7DEB786E099
:10248000E4EFF1E0DE01119601900D928A95E1F7FB
:10249000E090F601F090F7010091F8011091F90138
:1024A0001092F6011092F7011092F8011092F901C2
:1024B000E11003C0FF2009F45DC08091EF0190910D
:1024C000F0010E94F016AC019091F201992339F0CD
:1024D00020910A0130E02417350758F04BC02091B5
:1024E0000B018AE0289F900111242417350718F06A
:1024F00041C09F3F19F09F5F9093F201EE2061F081
:102500000E94CC101E1414F09FEF01C091E0989F20
:10251000902D11249093F601FF2061F00E94CC10C1
:102520001F1414F09FEF01C091E0989F902D11248B
:102530009093F7013091F6013323E1F02091F701F8
:102540002223C1F045EB3403C0011124992319F073
:102550009093F60103C081E08093F60135EB2303ED
:10256000C0011124992319F09093F70103C081E071
:102570008093F701011103C0112309F45DC080911C
:10258000ED019091EE010E94F016AC019091F101E5
:10259000992339F02091060130E02417350758F0CF
:1025A0004BC0209107018AE0289F90011124241735
:1025B000350718F041C09F3F19F09F5F9093F101DC
:1025C000002361F00E940B11101614F09FEF01C060
:1025D00091E0989F902D11249093F801112361F0C0
:1025E0000E940B11111614F09FEF01C091E0989F0B
:1025F000902D11249093F9013091F8013323E1F0EB
:102600002091F9012223C1F045EB3403C0011124CC
:10261000992319F09093F80103C081E08093F801A9
:1026200035EB2303C0011124992319F09093F9018C
:1026300003C081E08093F9018091F60181110BC004
:102640008091F701811107C08091F801811103C0C9
:102650008091F90181110E941612EB82FC820D8398
:102660001E8386E0FE013196A4EFB1E001900D9249
:102670008A95E1F726960FB6F894DEBF0FBECDBF60
:10268000DF91CF911F910F91FF90EF900895E4EFAC
:10269000F1E086E0DF011D928A95E9F71092F201E0
:1026A0001092F1011092F3010895CF93DF93EC01A2
:1026B000FB018281882309F43CC1C430FDE5DF07BA
:1026C00060F4CB3F9CE5D90788F49E0122503C453D
:1026D0002431310508F02EC109C0C236EDE5DE0710
:1026E00029F0C63AFDE5DF0709F024C10E94310C4C
:1026F0009093140280931302C1318CE5D80709F43A
:10270000C6C008F042C0C930ECE5DE0709F49BC042
:1027100000F5C5308CE5D80709F485C078F4C330DE
:10272000ECE5DE0709F478C008F07AC0C230DC4579
:1027300009F0F5C0809113028160EFC0C7309CE5BD
:10274000D90709F478C008F07AC08091130280613B
:10275000E4C0CD30FCE5DF0709F487C058F4CB3086
:102760009CE5D90709F479C008F07BC08091130279
:1027700088606FC0CF30FCE5DF0709F480C008F047
:1027800082C080911302877FC8C0CE3F9CE5D907E5
:1027900009F471C000F5C531FCE5DF0709F485C017
:1027A00068F4C3319CE5D90709F475C008F095C0F9
:1027B0000E94E805809113028F77AFC0CC3FFCE503
:1027C000DF07A9F108F054C0CB3FDC4509F0A7C0F2
:1027D0008091140240C0C230EDE5DE0709F489C0E3
:1027E00058F4C1158DE5D80709F45AC008F069C03E
:1027F0008091140282602FC0C236EDE5DE0709F435
:102800007CC0C63AFDE5DF0709F481C0C330DD4571
:1028100009F085C080E06EC08091130282607DC0A7
:102820008091130216C080911302886076C0809157
:10283000140282604FC08091130280626EC080914A
:10284000130280646AC00E94E805809113028068C8
:1028500064C0846062C081603DC0809113028E7F3D
:102860005CC0809113028D7F58C08091130216C006
:102870008091140218C0809114028D7F2BC080912A
:1028800013028F7E4AC0809113028F7D46C08091D3
:1028900013028F7B42C080911302877F8B7F3DC0E4
:1028A000809114028D7F8E7F15C08091130282FB70
:1028B000222720F991E0922790FB82F990FB83F97F
:1028C0002CC080911402982F909591708E7F892B47
:1028D00090FB81F98093140222C00E94E805809148
:1028E000130287FB222720F991E0922790FB87F9BA
:1028F00014C081E00E94C80C12C08091130284FBB6
:10290000222720F991E0922790FB84F906C080915C
:102910001302982F909590FB80F980931302809179
:102920001302909114020E94420C0E94E80580E07C
:1029300001C081E0DF91CF910895CF93DF9386317D
:102940009C4541F5EB010E943B0B982F8A81209119
:10295000020130910301882379F09A7A81E009F429
:1029600080E08093FA01911102C069E201C065E341
:10297000C9010E9430160AC08091FA01811102C07B
:1029800069E201C065E3C9010E9432160E947D0B15
:1029900080E001C081E0DF91CF9108950F931F93F4
:1029A000CF93DF93C42FD22FFC0182818823C9F0FB
:1029B0004093FD010E94D8169093FC018093FB0187
:1029C00080E28C0F883008F057C0C77081E001C0EA
:1029D000880FCA95EAF7DF91CF911F910F910C9460
:1029E00045038091FD01481330C08091FB01909117
:1029F000FC010E94F016883C910538F510E21D0F8D
:102A0000CD17B9F080E28C0F883040F4C77081E0B8
:102A100001C0880FCA95EAF70E944C03183028F5C8
:102A200081E09D2F977001C0880F9A95EAF70E9468
:102A30004503802F0E943C031830F0F4D77081E0EA
:102A400001C0880FDA95EAF70AC080E28C0F88305F
:102A500098F4C77081E001C0880FCA95EAF7DF914A
:102A6000CF911F910F910C944C03802FDF91CF9148
:102A70001F910F910C943C03DF91CF911F910F9107
:102A800008950F939C01CB01243F4CE5340731F1AD
:102A900088F4293DFCE53F07D9F02A3D4CE5340791
:102AA00079F1283D3C45A9F506E221EE41EE68EDBD
:102AB0007CE52BC0263FFCE53F07E1F0A8F0273F6F
:102AC0003C4539F507E225EE46EE67EF7CE51DC093
:102AD00007E225EE45EE69ED7CE517C006E221EE42
:102AE00040EE64EF7CE511C007E225EE44EE65EFB1
:102AF0007CE50BC006E221EE42EE66EF7CE505C008
:102B000008E221E045EE6AED7CE50E94CE1480E00B
:102B100008C0FC018281882319F01092FD0101C0D8
:102B200081E00F910895909383018093820108952D
:102B300090930302809302020895E0910202F091C3
:102B40000302309721F00190F081E02D099480E09C
:102B50000895E0910202F0910302309721F0028083
:102B6000F381E02D09940895E0910202F0910302AF
:102B7000309739F022E0DC012C930480F581E02DC0
:102B80000994089520910002309101022817390715
:102B900071F09093010280930002E0910202F091A3
:102BA0000302309721F00680F781E02D0994089503
:102BB0002091FE013091FF012817390771F09093A1
:102BC000FF018093FE01E0910202F0910302309731
:102BD00021F00084F185E02D09940895FC013296DE
:102BE00097E080E0915029F021912223D9F38F5F63
:102BF000F9CF0895662349F0FC0132960896219199
:102C0000621729F0E817F907D1F780E0089581E00D
:102C100008959C01FC0132969FEF80E04191461798
:102C200089F09F3F19F4411101C0982F8F5F8630C2
:102C3000A9F79F3F39F0F901E90FF11D97FDFA95CA
:102C40006283089508959C012A5F3F4FFC014281F1
:102C5000461301C01282019682179307B9F70895AF
:102C60000C9409160C942316029626E0FC0111928E
:102C70002A95E9F7089508950C943B1683E0809314
:102C800004020C943C16811102C081E001C082E074
:102C9000809304020C943C160C94431681E08093BC
:102CA00004020C943C160C944E1608950C94551680
:102CB0000C9456160C9455160C9455160C945516E7
:102CC0000E945C160E9444100E945A1680E00E94E6
:102CD000C90F811108C081E00E94C90F91E08111E4
:102CE00003C090E001C091E0892F089508951F92DC
:102CF0000F920FB60F9211248F939F93AF93BF93B0
:102D000080910502811113C08091190290911A02DD
:102D1000A0911B02B0911C024196A11DB11D809390
:102D2000190290931A02A0931B02B0931C02BF9148
:102D3000AF919F918F910F900FBE0F901F9018959C
:102D400080912102843031F10E942002109205020C
:102D500020E488E190E00FB6F894A8958093600095
:102D60000FBE2093600083B7817F846083BF83B7E9
:102D7000816083BF7894889583B78E7F83BF0FB6B9
:102D8000F894A8958091600088618093600010920B
:102D900060000FBE08950E94E8050C94240282E0B2
:102DA00084BD93E095BD9AEF97BD80936E00089522
:102DB0002FB7F8948091190290911A02A0911B02EA
:102DC000B0911C022FBF08952FB7F894609119029B
:102DD00070911A0280911B0290911C022FBF0895DE
:102DE0009C014FB7F8948091190290911A02A0911A
:102DF0001B02B0911C024FBF821B930B0895789465
:102E00001F920F920FB60F9211248F939F93AF933F
:102E1000BF938091190290911A02A0911B02B09168
:102E20001C020196A11DB11D8093190290931A02F4
:102E3000A0931B02B0931C02BF91AF919F918F9101
:102E40000F900FBE0F901F901895F89481E080931B
:102E5000E00080E28093D800E9ECF0E010828FE19E
:102E60009EE40197F1F700C000001DBA10926800BF
:102E70001CBC10BE1FBA10927A0010926E00109205
:102E80006F0010927100109272001082ECEBF0E073
:102E9000108214B817B81AB81DB810BA108215B835
:102EA00018B81BB81EB811BA0C94003F0895809151
:102EB00011020895089522E02093E9002FEF309148
:102EC000E800215035FD06C035ED3A95F1F70000D8
:102ED0002111F5CF2091E80025FF0BC040E050E024
:102EE00066E070E00E9485198091E8008E778093FB
:102EF000E8000895CF93DF9321E02093E9002FEFBE
:102F00003091E800215035FD06C035ED3A95F1F7D6
:102F100000002111F5CF2091E80025FF14C0EC013D
:102F200040E050E068E070E00E9485198091E80080
:102F30008E778093E80088E0FE01A9E0B2E001907E
:102F40000D928A95E1F7DF91CF9108958093060263
:102F5000709308026093070280912102843001F58A
:102F600082E08093E9008FEF9091E800815095FD19
:102F700006C095ED9A95F1F700008111F5CF80918B
:102F8000E80085FF0DC040E050E063E070E086E0BF
:102F900092E00E9485198091E8008E778093E80086
:102FA0000895BC0184E00C94A617BC0183E00C9446
:102FB000A61780912002811109C00E94161B0E9451
:102FC000731B8091E20084608093E2000895109268
:102FD000200208950C94531660911D0281E0611146
:102FE00001C080E00C943E169091210281E0943063
:102FF00009F080E060911D020C94431642E061EC00
:1030000081E00E948F1A42E261EC82E00E948F1AF6
:103010009091210281E0943009F080E060911D02DE
:103020000C944C1680912302833009F461C030F473
:10303000813071F0823009F49AC008958A3009F421
:1030400086C08B3009F46CC0893009F0A8C020C05C
:1030500080912202813A09F0A2C08091E800877F26
:103060008093E8008091260290912702892B21F419
:1030700068E089E092E003C060E080E090E070E00A
:103080000E94D0198091E8008B778093E800089522
:1030900080912202813209F082C0809126029091B3
:1030A0002702029708F07BC08091E800877F809319
:1030B000E8008091E80082FD05C080912102811125
:1030C000F8CF6DC02091F3008091F20090E0922B38
:1030D000029731F48091F100813011F0863021F4B3
:1030E0008091F100809311028091E8008B7753C0AA
:1030F00080912202813A09F052C08091260290917B
:103100002702892B09F04BC08091E800877F8093CC
:10311000E8008091E80080FFFCCF8091180136C064
:10312000809122028132D9F5809126029091270266
:10313000892BA9F58091E800877F8093E8000E94A1
:10314000C41A80912402809318010C94E8058091A0
:103150002202813221F58091E800877F8093E80088
:103160000E94C41A809125028093120208958091D2
:103170002202813AA1F48091E800877F8093E800E1
:103180008091E80080FFFCCF809112028093F100D3
:103190008091E8008E778093E8000C94C41A08951B
:1031A00084B7877F84BF0FB6F894A895809160009C
:1031B000886180936000109260000FBE90E080E80C
:1031C0000FB6F89480936100909361000FBE0C9449
:1031D0004E160E94161B0E94731BE2EEF0E08081E7
:1031E0008460808378940C94081E8CE091E00C94A9
:1031F0009815809121028530A9F4809121028530B3
:1032000079F40E94A01680911F028823B1F30E94D6
:103210006016882391F30E946F190E94E805EDCF94
:103220000C94CB16089508950C941619292F332762
:1032300023303105C9F060F42130310581F02230AE
:10324000310509F044C08BE390E020E231E043C057
:1032500021323105E1F02232310549F138C082E1F5
:1032600090E02BE531E037C099278130910549F096
:1032700028F0029761F5E0EFF0E005C0ECE1F1E045
:1032800002C0E8E0F1E0849190E09F0124C0611564
:10329000710541F061307105D1F489E090E02BE4D3
:1032A00031E019C089E090E022E331E014C06115FB
:1032B000710541F06130710551F48BE790E02DE626
:1032C00031E009C080E490E028EE31E004C080E005
:1032D00090E020E030E0FA0131832083089580E11E
:1032E00089BD82E189BD09B400FEFDCF8091D8007F
:1032F0008F7D8093D8008091E00082608093E00011
:103300008091E00081FDFCCF0895CF92DF92EF9293
:10331000FF920F931F93CF93DF93EC018B017A0100
:103320000E94E31A811133C0E114F10439F0F7016E
:1033300080819181081B190BC80FD91FC12CD12C7A
:103340000115110519F18091E80085FD16C08091E5
:10335000E8008E778093E800E114F10449F0F7016A
:1033600080819181C80ED91ED182C08285E00FC0B4
:103370000E94E31A882321F30AC089918093F10007
:1033800001501109FFEFCF1ADF0ADACF80E0DF9199
:10339000CF911F910F91FF90EF90DF90CF90089504
:1033A00020912802309129022617370748F061152D
:1033B000710539F42091E8002E772093E80001C0D0
:1033C000B901FC0120E06115710579F180912102BC
:1033D0008823F1F18530F1F18091E80083FD3CC054
:1033E0008091E80082FD2EC08091E80080FFEBCF45
:1033F0002091F3008091F20090E0922B611571050D
:1034000051F08830910538F421912093F1006150FA
:1034100071090196F3CF21E0089709F020E080912F
:10342000E8008E778093E800CECF2111CFCF0AC07D
:1034300080912102882361F0853061F08091E8005D
:1034400083FD0AC08091E80082FFF2CF80E00895FA
:1034500082E0089583E0089581E008952091280294
:10346000309129022617370748F06115710539F4A4
:103470002091E8002E772093E80001C0B901FC01FB
:1034800020E06115710591F180912102882309F4F2
:1034900040C0853009F43FC08091E80083FD3DC005
:1034A0008091E80082FD2FC08091E80080FFE9CF85
:1034B0002091F3008091F20090E0922B611571054C
:1034C00059F08830910540F424912093F100319611
:1034D000615071090196F2CF21E0089709F020E0D0
:1034E0008091E8008E778093E800CBCF2111CCCF7C
:1034F0000AC080912102882361F0853061F08091BB
:10350000E80083FD0AC08091E80082FFF2CF80E0EE
:10351000089582E0089583E0089581E00895982F4A
:10352000973068F59093E900981739F07091EC00A6
:103530002091ED005091F00003C0242F762F50E031
:1035400021FD02C09F5FECCF3091EB003E7F3093B6
:10355000EB003091ED003D7F3093ED003091EB00BA
:1035600031603093EB007093EC002093ED005093AA
:10357000F0002091EE0027FDE5CF80E008958F70E8
:103580008093E90081E008958091220287FF11C0B5
:103590008091E80082FD05C0809121028111F8CF61
:1035A00011C08091E8008B770BC0809121028823A5
:1035B00049F08091E80080FFF8CF8091E8008E7795
:1035C0008093E80008952091E4003091E50095E6AD
:1035D0004091EC00842F817040FF23C08091E8006F
:1035E00080FD1DC080912102882399F0853099F0DB
:1035F0008091EB0085FD11C04091E4005091E50001
:103600002417350729F3915011F09A01E1CF84E096
:10361000089582E0089583E0089581E0089580E0B0
:1036200008954091E80042FFDDCF08950E94841B79
:103630000E948C1BE0EEF0E0808181608083E8EDE9
:10364000F0E080818F77808319BCA7EDB0E08C918A
:103650008E7F8C9380818F7E8083109220020895CC
:103660000F931F93CF93DF930E94841B0E948C1BA8
:10367000C8EDD0E088818F778883888180688883CF
:1036800088818F7D888319BC1092210210921D02BF
:1036900010921F0210921E0200EE10E0F8018081CD
:1036A0008B7F808388818160888342E060E080E056
:1036B0000E948F1AE1EEF0E080818E7F8083E2EE3F
:1036C000F0E0808181608083808188608083F80160
:1036D00080818E7F8083888180618883DF91CF9114
:1036E0001F910F910895E8EDF0E080818F7E808337
:1036F000E7EDF0E080818160808384E082BF81E03B
:10370000809320020C94301BE8EDF0E080818E7FE6
:1037100080831092E20008951092DA001092E10086
:1037200008951F920F920FB60F9211242F933F937B
:103730004F935F936F937F938F939F93AF93BF93B9
:10374000EF93FF938091E10082FF0BC08091E20034
:1037500082FF07C08091E1008B7F8093E1000E948F
:10376000071E8091DA0080FF1FC08091D80080FF83
:103770001BC08091DA008E7F8093DA008091D9009F
:1037800080FF0DC080E189BD82E189BD09B400FEE2
:10379000FDCF81E0809321020E94D91705C019BC9A
:1037A000109221020E94E7178091E10080FF19C06A
:1037B0008091E20080FF15C08091E2008E7F8093AF
:1037C000E2008091E20080618093E2008091D80065
:1037D00080628093D80019BC85E0809321020E940A
:1037E000EC178091E10084FF30C08091E20084FFFB
:1037F0002CC080E189BD82E189BD09B400FEFDCF06
:103800008091D8008F7D8093D8008091E1008F7ED9
:103810008093E1008091E2008F7E8093E2008091AE
:10382000E20081608093E20080911D02882311F004
:1038300084E007C08091E30087FD02C081E001C001
:1038400083E0809321020E94F4178091E10083FFBE
:1038500029C08091E20083FF25C08091E100877F2D
:103860008093E10082E08093210210921D028091FA
:10387000E1008E7F8093E1008091E2008E7F809353
:10388000E2008091E20080618093E20042E060E02B
:1038900080E00E948F1A8091F00088608093F00091
:1038A0000E94EA17FF91EF91BF91AF919F918F9185
:1038B0007F916F915F914F913F912F910F900FBE2C
:1038C0000F901F9018951F920F920FB60F92112410
:1038D0002F933F934F935F936F937F938F939F9318
:1038E000AF93BF93CF93DF93EF93FF93C091E90022
:1038F000CF708091EC00D82FD17080FDD0E810926D
:10390000E9008091F000877F8093F00078940E9416
:10391000A71C1092E9008091F00088608093F0006D
:10392000CD2BCF70C093E900FF91EF91DF91CF9144
:10393000BF91AF919F918F917F916F915F914F91C7
:103940003F912F910F900FBE0F901F9018951F93CE
:10395000CF93DF93CDB7DEB7AA970FB6F894DEBF4B
:103960000FBECDBFE2E2F2E08091F100819322E050
:10397000EA32F207C9F70E9412188091E80083FF2B
:103980002EC18091220290912302492F50E04A30AB
:10399000510508F024C1FA01EE59FF4F0C94371E6F
:1039A000803821F0823809F01AC108C080911E02C7
:1039B00090911F02992389F082600FC080912602A6
:1039C0008F70873008F00BC18093E9008091EB0085
:1039D00085FB882780F91092E9009091E800977F95
:1039E0009093E8008093F1001092F100D1C0282F4D
:1039F0002D7F09F0F4C0882319F0823061F0EFC008
:103A000080912402813009F0EAC0933009F080E00F
:103A100080931F022EC08091240281112AC08091C0
:103A200026028F702FEF280F263008F0D8C0809321
:103A3000E9002091EB0020FF1CC0933021F480911D
:103A4000EB00806214C09091EB0090619093EB00CA
:103A500021E030E0A90102C0440F551F8A95E2F72A
:103A60004093EA001092EA008091EB008860809316
:103A7000EB001092E9008091E800877F8093E800D6
:103A80000E94C41AACC08111AAC0109124021F77F1
:103A90008091E3008078812B8093E3008091E8009F
:103AA000877F8093E8000E94C41A8091E80080FF1D
:103AB000FCCF8091E30080688093E300111102C085
:103AC00082E001C083E08093210289C08058823067
:103AD00008F085C080912402909125028C3D53E02E
:103AE000950779F583E08A838AE289834FB7F89452
:103AF000DE01139620E03EE051E2E32FF0E0509328
:103B00005700E49120FF03C0E295EF703F5FEF7034
:103B10008E2F90E0EA3010F0C79601C0C0968D93CA
:103B20009D932F5F243149F74FBF8091E800877F35
:103B30008093E8006AE270E0CE0101960E94D019FD
:103B400016C06091260270912702AE014F5F5F4F51
:103B50000E941419BC01892B09F441C09091E8001E
:103B6000977F9093E80089819A810E942E1A809114
:103B7000E8008B778093E80032C0803881F580912F
:103B8000E800877F8093E80080911D028093F10018
:103B90008091E8008E7772CF811121C0809124023C
:103BA0009091250299270297D4F48091E800877FAD
:103BB0008093E8008091240280931D020E94C41A21
:103BC00080911D02811106C08091E30087FD02C033
:103BD00081E001C084E0809321020E94FE17809161
:103BE000E80083FF0AC08091E800877F8093E800A7
:103BF0008091EB0080628093EB00AA960FB6F89458
:103C0000DEBF0FBECDBFDF91CF911F910895089504
:103C1000CF93809121028823A1F0C091E900CF7059
:103C20009091EC00892F817090FD80E8C82B109254
:103C3000E9008091E80083FD0E94A71CCF70C0932B
:103C4000E900CF91089597FB072E16F4009407D052
:103C500077FD09D00E943D1E07FC05D03EF49095EB
:103C600081959F4F0895709561957F4F0895EE0F50
:103C7000FF1F0590F491E02D0994AA1BBB1B51E195
:103C800007C0AA1FBB1FA617B70710F0A61BB70BCC
:103C9000881F991F5A95A9F780959095BC01CD0171
:103CA0000895FB01DC0104C08D910190801921F47D
:103CB00041505040C8F7881B990B0895F999FECFE1
:103CC00092BD81BDF89A992780B50895A8E1B0E02A
:103CD00042E050E00C94921E262FF999FECF92BD3F
:103CE00081BDF89A019700B4021639F01FBA20BDC1
:103CF0000FB6F894FA9AF99A0FBE08950396272FF3
:103D00000E946D1E0E946C1E252F0E946D1E242F86
:103D10000C946D1E0196272F0E946D1E0C946C1E34
:103D2000DC01CB01FC01F999FECF06C0F2BDE1BD7B
:103D3000F89A319600B40D9241505040B8F708956A
:043D4000F894FFCF25
:103D4400C800D501280850011E0A140157177A1714
:103D54005B17D517D1175A1701E200E900EA00B53D
:103D640000B600B700CD008301CC008A0192019413
:103D7400012102230224022502260227022A02B379
:103D840000B4006F007000818283E200E900EA0061
:103D9400B500B600B700CD008301CC008A019201C2
:103DA40094012102230224022502260227022A0268
:103DB400B300B4006F007000818283F7F6F1F5F46C
:023DC400F0000D
:00000001FF
